:100000000C9465020C94A9020C94A9020C94A90208
:100010000C94A9020C94A9020C94A9020C94A902B4
:100020000C94A9020C94A9020C94C50B0C94970C87
:100030000C94A9020C94A9020C94A9020C94A90294
:100040000C94A9020C9422210C94A9020C94A902EC
:100050000C94A9020C94C41A0C94A9020C94A90241
:100060000C94A9020C94A9020C94A9020C94A90264
:100070000C94A9020C94A9020C94A9020C94A90254
:100080000C94A9020C94A9020C94A9020C94A90244
:100090000C94A9020C94A9020C94A9020C94A90234
:1000A0000C94A9020C94A9020C94A902FC0C1E0D3C
:1000B000090E1E0D090E600D830D090ED80DEB0DF6
:1000C000D810D81006110611481184118413841316
:1000D0009C118413931293125E138413841372136E
:1000E0000000F0A12E004C002A00E1003581000044
:1000F0001E00140004001D7134004D001F001A0082
:1001000016001B00E1042A0020000800070006007A
:1001100050002C0021001500090019004F004A0072
:10012000220017000A000500000065745000015409
:100130000000007F0000E3004F0001540000007742
:100140000000E20023001C000B00110000002971D8
:10015000240018000D00100052004B0025000C0078
:100160000E00360051002800260012000F00370054
:100170002F002B00270013003382387130004E000F
:100180002D0031003478E500C100000001000100BD
:1001900001000100010000003A001E0220022202BC
:1001A000010001003B001F022102230201000100A7
:1001B0003C002F0226022F00010001003D0030020A
:1001C00027023000010001003E00310235003502F7
:1001D000000001000100010000000100000001001A
:1001E0000100010000000100000001003F0052007A
:1001F00051002402000001004000240021001E00E4
:10020000010001004100250022001F00370001000D
:1002100042002600230020002700010043002502A1
:100220002E0231002E0001004400450001000100B3
:1002300001000000010001000100010001000000B8
:1002400001000100010001000100010001000100A6
:10025000F2000100010001000100F000F1000100C6
:10026000F400010001000100F3000100F5000100AD
:100270000100010001000100000001000100010077
:100280000000010000000100010001000000010069
:100290000000010001000100010001000000010058
:1002A0000100010001000100A9000100010001009E
:1002B0000100AC00AA00B600010001000100AB0083
:1002C000A80001000100010001000100010001007F
:1002D00001000100AE00010001000000160345000E
:1002E000720067006F0044006F0078002000450036
:1002F0005A00000016034500720067006F004400BA
:100300006F007800200045005A0000000403090433
:1003100009026D00040100A0FA09040000010301B4
:100320000100092111010001223F00070581030896
:10033000000A090401000103010200092111010062
:1003400001224D000705820308000A09040200018A
:100350000300000009211101000122360007058376
:100360000308000A09040300010300000009211129
:100370000100012239000705840310000112011059
:100380000100000008EDFE07130100010200010555
:10039000010906A101050719E029E71500250195C6
:1003A0000875018102050819012905950575019156
:1003B000029501750391010507190029771500259C
:1003C00001957875018102C005010980A1018502AE
:1003D00016010026B7001A01002AB7007510950112
:1003E0008100C0050C0901A1018503160100269CAE
:1003F000021A01002A9C02751095018100C00501B6
:100400000902A1010901A100050919012905150029
:10041000250195057501810295017503810105018D
:10042000093009311581257F950275088106093843
:100430001581257F950175088106050C0A3802157E
:1004400081257F950175088106C0C005010906A1B7
:1004500001050719E029E7150025019508750181B7
:100460000295017508810105081901290595057591
:100470000191029501750391010507190029FF15E6
:100480000025FF950675088100C0000000000000EF
:100490000000000000010204060A0F17202C3A4A4F
:1004A0005D71879DB3C7DAE9F5FCFFFCF5E9DAC7B2
:1004B000B39D87715D4A3A2C20170F0A060402018A
:1004C0000000000000000000000011241FBECFEF5C
:1004D000DAE0DEBFCDBF04B603FE24C08091EE019A
:1004E0009091EF01A091F001B091F1018730904B14
:1004F000A740B04BB9F41092EE011092EF011092A8
:10050000F0011092F10114BE84B7877F84BF88E1A7
:100510000FB6F89480936000109260000FBEE0E088
:10052000FFE3099511E0A0E0B1E0E8ECF5E402C0DA
:1005300005900D92A433B107D9F711E0A4E3B1E01F
:1005400001C01D92AE3EB107E1F70E940B090C9469
:10055000E2220C94000061110BC0FC01828188230F
:1005600021F085EE0E946C0F03C085EE0E943410CE
:1005700080E090E0089508956091B1017091B2011A
:100580008091B3019091B4010E94F01956985E9841
:1005900025982D9826982E9827982F98813019F015
:1005A000823021F00895259A2D9A0895269A2E9A40
:1005B00008958CEB92E0892B11F00E94BC0280E040
:1005C00090E0089556985E9825982D9826982E9834
:1005D00027982F988FEF90E0909389008093880060
:1005E00090938B0080938A0090938D0080938C0071
:1005F000259A2D9A2FEF80E792E02150804090407D
:10060000E1F700C00000269A2E9A2FEF80E792E0D3
:10061000215080409040E1F700C00000279A2F9AB7
:100620002FEF80E792E0215080409040E1F700C03A
:10063000000025982D982FEF80E792E02150804010
:100640009040E1F700C0000026982E982FEF80E739
:1006500092E0215080409040E1F700C000002798D0
:100660002F9856985E9825982D9826982E9827981A
:100670002F98089589EA8093800089E08093810013
:1006800024982C983F988AB18F748AB96E98479AAB
:100690008BB1806B8BB9769A0E94E2028BEB92E071
:1006A000892B11F00E94BB0280E090E0089580E267
:1006B000809300018091340181110EC00E94A60335
:1006C00081E0809334012FEF83ED90E3215080404F
:1006D0009040E1F700C0000080E40E94AC038093EA
:1006E000000181112EC00E94D60380930001811168
:1006F00028C00E94D60380930001811122C08FE39D
:100700000E94D6038093000181111BC00E94CE037A
:1007100080E40E94AC0380930001811112C08CE040
:100720000E94D6038093000181110BC00E94D60362
:1007300080930001811105C08FE30E94D60380934E
:1007400000010E94CE038091000108951092B9002B
:100750008AE08093B800089594EA9093BC00909149
:10076000BC0097FFFCCF9091B900987F983021F0A2
:10077000903111F081E008958093BB0084E880936C
:10078000BC008091BC0087FFFCCF8091B900887FBE
:10079000883111F0803471F780E0089584E9809306
:1007A000BC008091BC0084FDFCCF08958093BB0009
:1007B00084E88093BC008091BC0087FFFCCF9091BF
:1007C000B900987F81E0983209F480E0089584E8C8
:1007D0008093BC008091BC0087FFFCCF8091BB0060
:1007E000089580910001811115C080E40E94AC033E
:1007F0008093000181110CC082E10E94D603809396
:100800000001811105C08FEF0E94D6038093000183
:100810000E94CE0384B1807F84B985B1807F85B981
:100820008AB1837F8AB98BB1837F8BB93E98469812
:1008300008950E945703809300010E94F10380B342
:100840008C7080BB81B3836F81BBE4E4F1E0A6E3ED
:10085000B1E011921D9281E0E235F807D1F78AE309
:1008600093E0892B11F00C943A030895BF92CF9234
:10087000DF92EF92FF920F931F93CF93DF938091BC
:100880000001882379F0809135018F5F80933501D5
:10089000811108C00E94570380930001811102C09A
:1008A0000E94E20206E311E0C0E0D0E0DD24D39430
:1008B00082E0C82EEE24E394F12CC73000F580913D
:1008C0000001811162C080E40E94AC0380930001AA
:1008D000811112C082E10E94D60380930001811130
:1008E0000BC0C7010C2E01C0880F0A94EAF780954F
:1008F0000E94D603809300010E94CE0346C0CA30F6
:10090000A1F028F4C83059F0C93061F005C0CC30EE
:1009100089F070F0CD3089F0209A289810C0219A83
:1009200029980DC0229A2A980AC0239A2B9807C0AA
:10093000529A01C0539A5B9802C03E9A4698E0EAE8
:10094000EA95F1F78FB1799960C092E081708D25B9
:10095000892B7C9B02C090E001C094E0892B7D9B99
:1009600002C090E001C098E0892B7E9B02C090E01D
:1009700001C090E1892B9FB19095991F9927991FEC
:100980009295990F907E892B0FC080910001811163
:1009900051C080E40E94AC03809300018823B9F128
:1009A000B12C0E94CE038B2DF8019081981719F07D
:1009B0008083C09201010E94F10321960F5F1F4FB7
:1009C000CE30D10509F079CF809101018823B1F0B3
:1009D000815080930101882339F08FE99FE00197CE
:1009E000F1F700C000000AC0A4E4B1E0E6E3F1E0E2
:1009F00081918D9391E0E434F907D1F789ED92E08C
:100A0000892BD1F00E94D90217C090E09FCF83E1DB
:100A10000E94D603809300018111C2CF81E40E941D
:100A2000AC03809300018111BBCF0E94E703B82E75
:100A3000B094B7CF80E0B8CF81E0DF91CF911F9124
:100A40000F91FF90EF90DF90CF90BF900895E82F27
:100A5000F0E0EC5BFE4F8081089508958B3B91059B
:100A600078F4883A910540F5853A9105D0F48430C0
:100A7000910508F0B1C08130910509F4ADC06BC09B
:100A8000803E910508F467C0883E910508F4A4C033
:100A90009C01205F31092031310508F05CC0906570
:100AA0000895853A910509F459C0863A910509F4EB
:100AB00058C083E890E40895883A910509F454C039
:100AC000893A910509F453C08A3A910509F452C054
:100AD0008B3A910509F451C08C3A910509F450C044
:100AE0008D3A910509F44FC0803B910509F44EC041
:100AF0008E3A910509F44DC08F3A910509F44CC026
:100B0000813B910509F44BC0823B910509F44AC031
:100B1000833B910509F449C0843B910509F448C021
:100B2000853B910509F447C0863B910509F446C011
:100B3000873B910509F445C0883B910509F444C001
:100B4000893B910509F443C08A3B910509F042C0F5
:100B50008AE296E4089580E090E0089581E890E4C8
:100B6000089582E890E4089582EE94E4089589EE71
:100B700094E408958AEE94E4089585EB94E408954E
:100B800086EB94E4089587EB94E408958CEC94E468
:100B900008958DEC94E4089583E895E408958AE837
:100BA00095E4089582E995E4089584E995E408952B
:100BB00081E296E4089583E296E4089584E296E45F
:100BC000089585E296E4089586E296E4089587E222
:100BD00096E4089580E094E40895089596E0799F5E
:100BE000F001112494E5899FE00DF11D1124E60F19
:100BF000F11DEE0FFF1FEC51FF4F85919491089569
:100C0000880F991F805A9040FC0185919491089516
:100C1000880F991F80529F4FFC01859194910895F0
:100C200026E0729FF001112444E5849FE00DF11D40
:100C30001124E60FF11DEE0FFF1FEC51FF4F259120
:100C40003491C9019A9581159F4110F4C901089505
:100C5000C90190528115904128F4C9019F700E94EA
:100C600008060895C90190538115904120F4C901E7
:100C70009927906C0895211580E5380769F40E9442
:100C8000A5139FEF24E34CE0915020404040E1F752
:100C900000C000000C94E91A213080E5380731F4D7
:100CA0008091CC0181608093CC010895C901905559
:100CB0008115904108F050C0832F99278F70992794
:100CC00081309105D9F4A9014370552702C0880FDE
:100CD000991F4A95E2F79C68A90164E0440F551FEB
:100CE0006A95E1F744275370842B952B73E0220F0C
:100CF000331F7A95E1F7207633271DC082309105A6
:100D000029F4922F8827816F906A08958330910586
:100D1000A9F4A9014370552781E090E002C0880F33
:100D2000991F4A95E2F79C6843E0220F331F4A95CA
:100D3000E1F7207E3770822B932B08950497F1F40E
:100D4000A9014370552781E090E002C0880F991FE8
:100D50004A95E2F79A68E8CFC9019057811590410A
:100D600020F4C9019F7090620895C90190588115BF
:100D7000904120F4C9019F70906A0895203E31058A
:100D8000E0F4203C310558F52133310509F470C0F9
:100D900048F42932310509F464C02A32310509F4D6
:100DA0006EC074C029333105F1F022383105D9F015
:100DB0002533310509F44EC069C0233E310589F160
:100DC00038F4203E3105C1F0223E3105E1F05EC02D
:100DD000263E310569F1273E3105A9F157C0C90109
:100DE0000E94000608958091DF0180FD02C081FF0E
:100DF0004DC080EE90E04BC08091DF0180FFF9CFC5
:100E000089E390E044C08091DF0182FF0EC08091B1
:100E1000DF0184FF03C080E090E039C083EE90E002
:100E200036C08091DF0182FFF2CF82EE90E02FC0CA
:100E30008091DF0183FF0BC08091DF0184FDEBCF48
:100E400087EE90E024C08091DF0183FFF5CF86EE2E
:100E500090E01DC08091DF0185FF07C089E290E02E
:100E600016C08091DF0185FFF9CF85E390E00FC0C8
:100E70008091DF0186FF07C08AE290E008C0809180
:100E8000DF0186FFF9CF81E390E001C0C9010E9434
:100E90002E0508950895809162010895CF93DF9300
:100EA00000D01F92CDB7DEB72091E501243019F5AF
:100EB00023E029839B838A832093E9008FEF90911D
:100EC000E800815095FD06C095ED9A95F1F7000078
:100ED0008111F5CF8091E80085FF0DC040E050E022
:100EE00063E070E0CE0101960E94B8098091E800AD
:100EF0008E778093E8000F900F900F90DF91CF9145
:100F00000895CF93DF9300D01F92CDB7DEB7209125
:100F1000E501243021F522E029839B838A8383E045
:100F20008093E9008FEF9091E800815095FD06C015
:100F300095ED9A95F1F700008111F5CF8091E800C9
:100F400085FF0DC040E050E063E070E0CE01019607
:100F50000E94B8098091E8008E778093E8000F9096
:100F60000F900F90DF91CF9108952091E5012430EB
:100F7000F1F422E02093E9002FEF3091E8002150B6
:100F800035FD06C035ED3A95F1F700002111F5CF9A
:100F90002091E80025FF0BC040E050E065E070E0E4
:100FA0000E94B8098091E8008E778093E800089548
:100FB000CF93DF93EC018091E501843009F046C0C6
:100FC00090910C019923D9F090910D019923B9F0DA
:100FD0008093E9008FEF9091E800815095FD06C065
:100FE00095E19A95F1F700008111F5CF8091E80025
:100FF00085FF2CC040E050E060E170E017C081E068
:101000008093E9008FEF9091E800815095FD06C034
:1010100095ED9A95F1F700008111F5CF8091E800E8
:1010200085FF14C040E050E068E070E0CE010E940F
:10103000B8098091E8008E778093E80080E1FE0196
:10104000A2E5B1E001900D928A95E1F7DF91CF9191
:1010500008958091E401811109C00E944A0B0E9409
:10106000A70B8091E20084608093E20008951092C3
:10107000E401089508950C940F210E94801A0E94A3
:1010800015210E94440E0C944A0742E061EC81E075
:101090000E94C40A42E061EC82E00E94C40A42E07D
:1010A00061EC83E00E94C40A42E161EC84E00C94AC
:1010B000C40A8091E701833009F455C030F48130CF
:1010C00071F0823009F48EC008958A3009F47AC034
:1010D0008B3009F460C0893009F09CC020C0809139
:1010E000E601813A09F096C08091E800877F8093FD
:1010F000E8008091EA019091EB01892B21F060E0FA
:1011000080E090E003C060E182E591E070E00E9441
:10111000010A8091E8008B778093E8000895809120
:10112000E601813209F076C08091EA019091EB01ED
:10113000009719F0039709F06DC08091E800877F50
:101140008093E8008091E80082FD05C08091E50170
:101150008111F8CF5FC08091F1008093620180918E
:10116000E8008B7753C08091E601813A09F052C0C4
:101170008091EA019091EB01892B09F04BC080919D
:10118000E800877F8093E8008091E80080FFFCCF33
:1011900080910C0136C08091E6018132D9F58091B1
:1011A000EA019091EB01892BA9F58091E800877FF6
:1011B0008093E8000E94F90A8091E80180930C0175
:1011C0000C94A5138091E601813221F58091E8000D
:1011D000877F8093E8000E94F90A8091E90180935B
:1011E000630108958091E601813AA1F48091E800BD
:1011F000877F8093E8008091E80080FFFCCF80919A
:1012000063018093F1008091E8008E778093E8007D
:101210000C94F90A089584B7877F84BF88E10FB6DC
:10122000F89480936000109260000FBE90E080E818
:101230000FB6F89480936100909361000FBE0E94F6
:10124000930E0E944A0B0E94A70B8091E2008460DB
:101250008093E20078940E94220E0E94950E82E014
:1012600091E00E943F0E0E94FD208091E5018530B3
:1012700069F40E94431A8091E3018823B1F30E942C
:101280006B1A882391F30E94A209EFCF0E949B0E54
:10129000ECCF292F332723303105A9F06CF421300E
:1012A000310509F442C02230310509F043C08DE612
:1012B00090E020E133E042C021323105C9F0223212
:1012C000310519F137C099278130910541F08230FD
:1012D000910541F0892B71F5ECE0F3E005C0E4EFF6
:1012E000F2E002C0ECEDF2E0849190E09F0126C0B4
:1012F000643000F5E62FF0E0EE0FFF1FEE5DFE4FCD
:101300002081318189E090E019C0643098F4E62FA3
:10131000F0E0DF01AA0FBB1FA65EBE4F2D913C91EE
:10132000EA5EFE4F808190E009C082E190E02DE707
:1013300033E004C080E090E020E030E0FA01318347
:101340002083089580E189BD82E189BD09B400FE52
:10135000FDCF8091D8008F7D8093D8008091E000F0
:1013600082608093E0008091E00081FDFCCF0895D1
:10137000CF92DF92EF92FF920F931F93CF93DF9361
:101380007C018B01EA010E941A0B811131C0209768
:1013900031F088819981081B190BE80EF91EC12CC8
:1013A000D12C0115110519F18091E80085FD14C0BB
:1013B0008091E8008E778093E800209741F0888143
:1013C00099818C0D9D1D9983888385E011C00E94B1
:1013D0001A0B882331F30CC0F70181917F018093B0
:1013E000F10001501109FFEFCF1ADF0ADACF80E0D8
:1013F000DF91CF911F910F91FF90EF90DF90CF90F1
:1014000008952091EC013091ED012617370748F03F
:101410006115710539F42091E8002E772093E800DA
:1014200001C0B901FC0120E061157105B9F180919D
:10143000E501882309F440C0853009F43FC080915C
:10144000E80083FD3DC08091E80082FF06C08091E6
:10145000E80082FF26C080E008958091E80080FFC8
:10146000E3CF2091F3008091F20090E0922B611580
:10147000710551F08830910538F421912093F100E5
:10148000615071090196F3CF21E0089709F020E03F
:101490008091E8008E778093E800C6CF2111C7CFF6
:1014A000D6CF8091E501882339F0853039F08091DD
:1014B000E80083FFCCCF04C082E0089583E0089564
:1014C00081E008952091EC013091ED012617370756
:1014D00048F06115710539F42091E8002E772093CA
:1014E000E80001C0B901FC0120E061157105C1F1FE
:1014F0008091E501882309F441C0853009F440C09A
:101500008091E80083FD3EC08091E80082FF06C024
:101510008091E80082FF27C080E008958091E80074
:1015200080FFE3CF2091F3008091F20090E0922BB6
:101530006115710559F08830910540F4249120938C
:10154000F1003196615071090196F2CF21E00897C0
:1015500009F020E08091E8008E778093E800C5CF05
:101560002111C6CFD5CF8091E501882339F0853090
:1015700039F08091E80083FFCBCF04C082E008956A
:1015800083E0089581E00895982F973058F590935F
:10159000E900981739F07091EC002091ED0050911E
:1015A000F00003C0242F762F50E021FF19C03091A6
:1015B000EB003E7F3093EB003091ED003D7F3093A8
:1015C000ED003091EB0031603093EB007093EC0054
:1015D0002093ED005093F0002091EE0027FF07C00C
:1015E0009F5FD3CF8F708093E90081E0089580E002
:1015F00008958091E60187FD05C08091E80080FF95
:101600000EC012C08091E80082FD05C08091E50106
:101610008111F8CF08958091E8008B7708C0809100
:10162000E5018111EACF08958091E8008E778093DB
:10163000E80008958091E4009091E50045E620914E
:10164000EC0020FF21C02091E80020FD21C0209166
:10165000E501222389F0253089F02091EB0025FD5A
:101660000FC02091E4003091E5002817390739F3C5
:10167000415041F0C901E3CF82E0089583E008952D
:1016800081E0089584E008952091E80022FFDFCFF3
:1016900080E008950E94B80B0E94C00BE0EEF0E0DD
:1016A000808181608083E8EDF0E080818F778083A6
:1016B00019BCA7EDB0E08C918E7F8C9380818F7EDA
:1016C00080831092E40108950F931F93CF93DF93CB
:1016D0000E94B80B0E94C00BC8EDD0E088818F77C4
:1016E000888388818068888388818F7D888319BCFE
:1016F0001092E5011092E1011092E3011092E201D3
:1017000000EE10E0F80180818B7F8083888181600A
:10171000888342E060E080E00E94C40AE1EEF0E0ED
:1017200080818E7F8083E2EEF0E080818160808323
:10173000808188608083F80180818E7F80838881AA
:1017400080618883DF91CF911F910F910895E8ED1B
:10175000F0E080818F7E8083E7EDF0E08081816022
:10176000808384E082BF81E08093E4010C94640B69
:10177000E8EDF0E080818E7F80831092E200089592
:101780001092DA001092E10008951F920F920FB6A6
:101790000F9211242F933F934F935F936F937F93F7
:1017A0008F939F93AF93BF93EF93FF938091E1004B
:1017B00082FF0BC08091E20082FF07C08091E100B0
:1017C0008B7F8093E1000E94210E8091DA0080FFE0
:1017D0001FC08091D80080FF1BC08091DA008E7FEF
:1017E0008093DA008091D90080FF0DC080E189BD2F
:1017F00082E189BD09B400FEFDCF81E08093E5015F
:101800000E94290805C019BC1092E5010E94370802
:101810008091E10080FF19C08091E20080FF15C037
:101820008091E2008E7F8093E2008091E2008061EF
:101830008093E2008091D80080628093D80019BC28
:1018400085E08093E5010E943B088091E10084FFE0
:1018500030C08091E20084FF2CC080E189BD82E12C
:1018600089BD09B400FEFDCF8091D8008F7D8093A3
:10187000D8008091E1008F7E8093E1008091E200AA
:101880008F7E8093E2008091E20081608093E2008D
:101890008091E101882311F084E007C08091E3008A
:1018A00087FF02C083E001C081E08093E5010E94D0
:1018B0003D088091E10083FF29C08091E20083FF11
:1018C00025C08091E100877F8093E10082E08093D2
:1018D000E5011092E1018091E1008E7F8093E100AB
:1018E0008091E2008E7F8093E2008091E20080612F
:1018F0008093E20042E060E080E00E94C40A8091B0
:10190000F00088608093F0000E943A08FF91EF9108
:10191000BF91AF919F918F917F916F915F914F9107
:101920003F912F910F900FBE0F901F9018951F920F
:101930000F920FB60F9211242F933F934F935F9303
:101940006F937F938F939F93AF93BF93CF93EF93B7
:10195000FF93C091E900CF708091EC001092E900F4
:101960008091F000877F8093F00078940E94D30CE0
:101970001092E9008091F00088608093F000C0939D
:10198000E900FF91EF91CF91BF91AF919F918F911E
:101990007F916F915F914F913F912F910F900FBE6B
:1019A0000F901F9018951F93CF93DF93CDB7DEB79D
:1019B000AA970FB6F894DEBF0FBECDBFE6EEF1E0FA
:1019C0008091F100819321E0EE3EF207C9F70E9479
:1019D00059088091E80083FF1CC12091E6013091F5
:1019E000E701832F90E08A30910508F012C1FC01D5
:1019F000EA5AFF4F0C949722203881F0223809F0E0
:101A000008C18091EA018F708093E9008091EB001A
:101A100085FB882780F91092E90006C08091E201D9
:101A20009091E301911182609091E800977F9093EB
:101A3000E8008093F1001092F100C5C0822F8D7FE5
:101A400009F0E7C0222319F0223061F0E2C0809152
:101A5000E801813009F0DDC0333009F080E0809387
:101A6000E30128C08091E801811124C02091EA019E
:101A70002F7009F4CEC02093E9008091EB0080FF25
:101A800019C08091EB00333011F4806211C0806185
:101A90008093EB0081E090E0022E01C0880F0A9451
:101AA000EAF78093EA001092EA008091EB008860E8
:101AB0008093EB001092E9008091E800877F86C058
:101AC0002111A7C01091E8011F778091E300807871
:101AD000812B8093E3008091E800877F8093E8006A
:101AE0000E94F90A8091E80080FFFCCF8091E3001A
:101AF00080688093E300112311F083E001C082E04D
:101B00008093E50186C02058223008F082C0809181
:101B1000E8019091E9018C3D23E0920779F583E09B
:101B20008A838AE289834FB7F894DE01139620E016
:101B30003EE051E2E32FF0E050935700E49120FFA4
:101B400003C0E295EF703F5FEF708E2F90E0EA30B8
:101B500010F0C79601C0C0968D939D932F5F2431DE
:101B600049F74FBF8091E800877F8093E8006AE2E1
:101B700070E0CE0101960E94010A14C0AE014F5FD1
:101B80005F4F6091EA010E944909009709F441C042
:101B90002091E800277F2093E800BC0189819A8189
:101BA0000E94620A8091E8008B778093E80031C040
:101BB000203879F58091E800877F8093E800809154
:101BC000E1018093F1008091E8008E778093E80036
:101BD0000E94F90A1EC021111CC09091E8019230A8
:101BE000C0F48091E800877F8093E8009093E10142
:101BF0000E94F90A8091E101811104C08091E30003
:101C000087FF02C084E001C081E08093E5010E946B
:101C100045088091E80083FF0AC08091E800877F33
:101C20008093E8008091EB0080628093EB00AA969D
:101C30000FB6F894DEBF0FBECDBFDF91CF911F91DD
:101C400008950895CF938091E5018823B1F08091A4
:101C5000E9008F709091EC0090FF02C090E801C005
:101C600090E0C92FC82B1092E9008091E80083FD15
:101C70000E94D30CCF70C093E900CF910895909348
:101C80006901809368010895E0916801F09169010C
:101C9000309721F00190F081E02D099480E00895C3
:101CA000E0916801F0916901309721F00280F381A1
:101CB000E02D09940895E0916801F0916901309751
:101CC00021F00480F581E02D0994089520916601AA
:101CD000309167018217930771F0909367018093A9
:101CE0006601E0916801F0916901309721F006806A
:101CF000F781E02D099408952091640130916501E8
:101D00008217930771F09093650180936401E091CD
:101D10006801F0916901309721F00084F185E02D90
:101D20000994089508950C94920E0E94861A0E94B8
:101D300019040C944C1BCF92DF92EF92FF920F93F9
:101D40001F93CF93DF93CDB7DEB72B970FB6F894E1
:101D5000DEBF0FBECDBF0E9436043BE6E32E31E06E
:101D6000F32E00E010E0C02E802F0E942705F7011F
:101D7000D1907F01D826B1F40F5F1F4F0E301105AF
:101D800091F78FEF89838A831B820E948F1A81606B
:101D9000782F9D838C8349815A816B818D810E942C
:101DA0003E0F41C09091CC0191FF04C08B870E94EF
:101DB0002D058B8520E030E04D2D50E0922FBA01AB
:101DC000022E02C0759567950A94E2F760FF25C060
:101DD0002E83CF82EE24E394F12C02C0EE0CFF1C84
:101DE0009A95E2F790E08E219F2121E0892B09F45A
:101DF00020E028870E948F1A8160782F9A87898730
:101E00004E815F8168858A850E943E0FF801E55901
:101E1000FE4F80818E25808306C02F5F3F4F263086
:101E2000310561F6A9CF0E94301E10916A010E940F
:101E3000440E1817A1F00E94440E80936A012B965D
:101E40000FB6F894DEBF0FBECDBFDF91CF911F91CB
:101E50000F91FF90EF90DF90CF900C944A072B9654
:101E60000FB6F894DEBF0FBECDBFDF91CF911F91AB
:101E70000F91FF90EF90DF90CF900895CF93DF9375
:101E8000CDB7DEB72B970FB6F894DEBF0FBECDBF30
:101E90004F83588769877A878B87DE01119686E0A2
:101EA000FD0111928A95E9F785E0FE0137960190D0
:101EB0000D928A95E1F749815A816B817C818D81F0
:101EC0009E810E9471162B960FB6F894DEBF0FBE4E
:101ED000CDBFDF91CF910895CF93C82F882309F408
:101EE000C1C0823859F40E94440E81FDBBC089E311
:101EF0000E9410190E94CA1989E30CC0833879F432
:101F00000E94440E80FDAEC083E50E9410190E941D
:101F1000CA1983E50E945019CF910C94CA198438CC
:101F200059F40E94440E82FD9DC087E40E9410195E
:101F30000E94CA1987E4EECF8CEF8C0F813A48F4E7
:101F40008C2F0E94652081118DC08C2F0E9410194A
:101F5000E3CF80E28C0F883048F4C77081E001C085
:101F6000880FCA95EAF70E949119D6CF8BE58C0F9E
:101F7000833078F4C53A29F0C63A31F482E890E02B
:101F800005C081E890E002C083E890E0CF910C9416
:101F9000660E88E58C0F833108F064C0C83A39F1C9
:101FA000C93A41F1CA3A49F1CB3A51F1CC3A59F127
:101FB000CD3A61F1C03B69F1CE3A71F1CF3A79F196
:101FC000C13B81F1C23B89F1C33B91F1C43B99F123
:101FD000C53BA1F1C63BA9F1C73BB1F1C83BB9F183
:101FE000C93BC1F1CA3BC9F58AE292E038C082EE32
:101FF00090E035C089EE90E032C08AEE90E02FC0CC
:1020000085EB90E02CC086EB90E029C087EB90E058
:1020100026C08CEC90E023C08DEC90E020C083E8DB
:1020200091E01DC08AE891E01AC082E991E017C0F2
:1020300084E991E014C081E292E011C083E292E071
:102040000EC084E292E00BC085E292E008C086E216
:1020500092E005C087E292E002C080E090E0CF917C
:102060000C947C0ECF910895882309F44BC08238DC
:1020700059F40E94440E81FF45C089E30E94101963
:102080000E94CA1989E30CC0833871F40E94440E7F
:1020900080FF38C083E50E9410190E94CA1983E5A9
:1020A0000E9450190C94CA19843859F40E94440EA5
:1020B00082FF28C087E40E9410190E94CA1987E491
:1020C000EFCF9CEF980F913A58F390E2980F983029
:1020D00050F4877091E001C0990F8A95EAF7892F33
:1020E0000E949719DFCF9BE5980F933020F480E092
